:10000000B201C8280408A700891009100910831636
:100010008910091009100F30880583122708B218BB
:100020002F283A30A10098308E203330A60043208C
:100030001330A10088308E20432064308D2043206F
:1000400064308D202230A600432028302E200C3032
:100050002E2006302E20B21427082F283214A60096
:10006000321C3D280910033C031C42284220073063
:10007000A100D0308E20031408003214FE3C031976
:10008000C3280914321C321089140F308805260841
:10009000F03988048910A60E3218432832308D209A
:1000A00003140800B31329080319B3170530A80077
:1000B0002730A300103068200330A300E830682008
:1000C000A30164306820A3010A30682024086F2847
:1000D000A2002508A1002408A000A2202008A0005A
:1000E000A8030319B3132908031979282802031850
:1000F00008002008031DB313B31B0800303EBE28C0
:10010000A301A200FF30A207031CA307031CC328FE
:100110000330A100DF308E208228A101E83EA0003C
:10012000A109FC30031C9728A00703189428A007F6
:100130006400A10F942820189D28A01CA12800006D
:10014000A1280800A501A4011030A600210DA40DCE
:10015000A50D2208A4022308031C230FA5020318DF
:10016000B8282208A40723080318230FA5070310A3
:10017000A00DA10DA60BA6282008C32884003108D5
:100180008A0030088200831303138312640008007E
:10019000831604309F0083120911831609116430FD
:1001A00083128A01802083160F3086008312860115
:1001B000BA010608B800FE308A01032001308A0126
:1001C000032054308A0103206F308A0103206E30EF
:1001D0008A01032020308A010320A9013808A400E5
:1001E000A5010230B000B1018A01522020308A01FD
:1001F000032048308A01032041308A010320523015
:100200008A01032046308A01032020308A0103201E
:1002100020308A0103203A088A01032028308A010D
:10022000802064003808073C8A110A12031D1A292D
:0E0230004130BA008A01D92863008A011C29D6
:02400E00753DFE
:00000001FF
